:100000007AC0000093C0000091C000008FC00000C3
:100010008DC000008BC0000089C0000087C00000B8
:1000200085C0000083C0000081C00000C9C200007C
:100030008EC100007BC0000079C0000077C00000C6
:1000400075C0000073C0000071C000006FC00000E8
:100050006DC000006BC0000069C00000D6C2000087
:1000600065C0000063C0000061C000005FC0000008
:100070005DC000000C035B007300650072005D0052
:1000800000000E035B00700072006F0064005D00F2
:1000900000000C035B006D00660067005D0000005F
:1000A0000403090409021200010100C0320904001E
:1000B0000000FF0101001201000000000040CDAB74
:1000C00003F0CDAB010203010000000000010000BD
:1000D000B6001200020000A4001200030000A000FD
:1000E000040103090492000C0203090482000E03B8
:1000F00003090474000C11241FBECFEFD4E0DEBF4F
:10010000CDBF11E0A0E0B1E0E4ECF8E002C0059062
:100110000D92A833B107D9F711E0A8E3B1E001C00F
:100120001D92A934B107E1F7FFD2CAC369CF282FC6
:10013000579898E080E05598880F4F998160559ABC
:100140009150C9F7211101C0579A5598559A57985F
:10015000089598E087FF02C0579801C0579A880F0A
:100160005598559A9150B1F75798559889B1559A25
:10017000881F8827881F0895579A559A5598579829
:100180000895579A559A0895EF92FF921F93CF932F
:10019000DF931F92CDB7DEB77C01F3DF82E5D9DFB5
:1001A00083E9D7DFE9DFEDDF81E0C1DF8983E4DFC9
:1001B000898180FFF2CF8FEFE81AF80A10E0E1DFC3
:1001C00082E5C7DF812F880F8C5E806AC2DFD4DFB3
:1001D000D8DF83E5BEDF80E0AADFF70131978083B7
:1001E00081E0A5DFF7018083C7DF1F5FF2E0EF0E3C
:1001F000F11C143021F70F90DF91CF911F91FF90E8
:10020000EF9008951F93CF93DF931F92CDB7DEB782
:10021000182F6983B6DF82E59CDF812F8F71806A9A
:1002200098DF6981862F95DF0F90DF91CF911F9125
:10023000A3CFCF93C82F81E0E5DF6EEF83E0E2DF4D
:100240006C2F8FE0CF91DECF8091E80080FFFCCF54
:100250000895FC0140812FE9240F263038F4242F23
:10026000332727FD30952755310902C020E030E0C3
:100270005FEB540F563030F4242F332727FD309591
:100280002753310950ED540F5A3030F4242F3327BF
:1002900027FD30952053310944E0220F331F4A9542
:1002A000E1F7FC0181819FE9980F963040F4482FD7
:1002B000552747FD509547555109242B352B9FEB6A
:1002C000980F963040F4482F552747FD50954753D7
:1002D0005109242B352B90ED980F9A3030F4992743
:1002E00087FD9095C097282B392B822F08959091E8
:1002F000C80095FFFCCFEFE3FFE13197F1F700C0B5
:1003000000008093CE000895CF93C82F982F929528
:100310009F709A3010F087E501C080E3890FE7DF16
:100320008C2F8F70282F30E02A30310514F0895A35
:1003300001C0805DCF91DBCFCF93DF93EC0189913A
:10034000882311F0D4DFFBCFDF91CF9108951F9266
:100350000F920FB60F9211240F931F932F933F9379
:100360004F935F936F937F938F939F93AF93BF93BD
:10037000EF93FF93CF93DF93CDB7DEB72897DEBF20
:10038000CDBF1092E9008091E80083FFFBC09091FF
:10039000F1008091F1000091F1002091F10010E056
:1003A000122B4091F1003091F1002091F100A091C9
:1003B000F10052EF5093E800863009F048C050E059
:1003C000532B36E08CEC90E0FC0165917491601742
:1003D000710739F4FC0132966591749164177507C1
:1003E00021F00796315081F7CDC0FC01349645913C
:1003F0005491FC013696849130E03A2B2F3F310521
:1004000019F010F02FEF30E0281708F4822F3EEF9C
:100410009091E800292F2570D9F392FDB6C0982F4E
:10042000813408F090E4FA01292F222331F06491FD
:100430006093F10021503196F8CF490F511D891B6F
:100440003093E8008111E4CF903411F39EC08530E1
:1004500041F48EEF8093E800F7DE00680093E3003C
:1004600094C0893079F591118DC0009348018EEFC9
:100470008093E80041E088EC90E04093E9009C0123
:100480002F5F3F4FFC0154915093EB00552361F0D7
:10049000F90124912093EC009C012D5F3F4FFC015A
:1004A000329684918093ED004F5F453011F0C90181
:1004B000E4CF8EE18093EA001092EA0082E080931C
:1004C000470163C0883049F4903809F05BC0BCDE56
:1004D000809148018093F10007C0811109C0B4DE0A
:1004E0001092F1001092F1008EEF8093E8004DC061
:1004F000843A09F047C081E080934601602F6095FF
:10050000812F837096DECE0101963EDE9DDE8A81CC
:100510008093F10089818093F1008C818093F100B8
:100520008B818093F1008E818093F1008D81809387
:10053000F10088858093F1008F818093F1008EEF28
:100540008093E80084B1806E84B987B1806C87B9EC
:1005500017FF02C02D9A01C02D9816FF02C02E9AD7
:1005600001C02E9815FF02C02F9A01C02F9814FFCA
:1005700002C0479A01C0479813FF02C0469A05C0BF
:10058000469803C081E28093EB0028960FB6F8945A
:10059000DEBF0FBECDBFDF91CF91FF91EF91BF9135
:1005A000AF919F918F917F916F915F914F913F910B
:1005B0002F911F910F910F900FBE0F901F901895C4
:1005C0001F920F920FB60F9211248F939F938091D9
:1005D000E1001092E10083FF11C01092E90081E078
:1005E0008093EB001092EC0092E39093ED0098E082
:1005F0009093F00010924801809347019F918F9152
:100600000F900FBE0F901F9018951F920F920FB66C
:100610000F921124FF920F931F932F933F934F93A9
:100620005F936F937F938F939F93AF93BF93EF935A
:10063000FF93CF93DF931F92CDB7DEB78091CE00AB
:10064000898380914501882309F457C08091420134
:10065000909143018A30910560F49C012F5F3F4FD8
:1006600030934301209342012981FC01E85CFE4F55
:10067000208389818A3021F089818E3209F03DC042
:100680008091420190914301079799F588E391E0A9
:10069000E0DD082F8AE391E0DCDDF82E8CE391E0C9
:1006A000D8DD182F6F2D6095802F8370C2DD84B147
:1006B000806E84B987B1806C87B914FF02C02D9A0F
:1006C00001C02D9813FF02C02E9A01C02E9812FF70
:1006D00002C02F9A01C02F9811FF02C0479A01C093
:1006E000479810FF02C0469A01C0469881E0809367
:1006F000440110924301109242010F90DF91CF917B
:10070000FF91EF91BF91AF919F918F917F916F91E9
:100710005F914F913F912F911F910F91FF900F90FB
:100720000FBE0F901F901895CF93DF93CDB7DEB714
:1007300029970FB6F894DEBF0FBECDBFF89481E0C5
:100740008AB9789480E880936100109261008FEFFD
:100750008093470180EA8093D8001092630086E07E
:1007600089BD09B400FEFDCF80E88093D8001092C7
:10077000E0008CE08093E2008FEC90E09093CD005D
:100780008093CC0082E08093C80088E98093C90000
:1007900086E08093CA00539A3A9A42988FE39CE984
:1007A0000197F1F700C00000429A9FEF23EC89E027
:1007B000915020408040E1F700C0000080E091E0CF
:1007C000BBDD9FEF23EC89E0915020408040E1F7B2
:1007D00000C000008BE091E0AFDD9FEF23EC89E0EB
:1007E000915020408040E1F700C0000080E191E09E
:1007F000A3DD9FEF23EC89E0915020408040E1F79A
:1008000000C000008CE291E097DD78949FEF23EC2C
:1008100089E0915020408040E1F700C0000081E075
:100820008093450105E010E08BB18F758BB98AB1DB
:100830008F758AB9A6DC82E58CDC89879DDC898589
:10084000882361F0015011090115110569F08FE34A
:100850009CE90197F1F700C00000E6CF6BE080E073
:10086000D1DC65ED8AE0E5DC809146018111FECFA7
:10087000809144018823E1F38FE19EE40197F1F731
:1008800000C00000CE0101967FDC8A813DDD8981B8
:100890003BDD80E22CDD8C8137DD8B8135DD80E234
:1008A00026DD8E8131DD8D812FDD80E220DD8885A2
:1008B0002BDD8F8129DD80E21ADD8AE018DDD4CFBF
:0408C000F894FFCFDA
:1008C40041542B52657365740D0A0041540D0A009E
:1008D40041542B4E414D45526F79436F6C6F727387
:1008E400526F79436F6C6F72730D0A0041542B522F
:0808F4004F4C45300D0A0000D5
:00000001FF
